:101800001AC135C134C133C132C131C130C129C25D
:101810002EC12DC12CC12BC12AC129C128C127C16C
:1018200026C125C1EBC123C1A9C121C120C11FC14E
:101830001EC11DC11CC10000211042206330844024
:10184000A550C660E770088129914AA16BB18CC18F
:10185000ADD1CEE1EFF13112100273325222B55206
:101860009442F772D662399318837BB35AA3BDD3DF
:101870009CC3FFF3DEE36224433420040114E664D6
:10188000C774A44485546AA54BB528850995EEE52F
:10189000CFF5ACC58DD55336722611163006D776E6
:1018A000F6669556B4465BB77AA719973887DFF77F
:1018B000FEE79DD7BCC7C448E5588668A7784008AE
:1018C000611802282338CCC9EDD98EE9AFF94889CF
:1018D00069990AA92BB9F55AD44AB77A966A711A46
:1018E000500A333A122AFDDBDCCBBFFB9EEB799B1F
:1018F000588B3BBB1AABA66C877CE44CC55C222C96
:10190000033C600C411CAEED8FFDECCDCDDD2AAD6E
:101910000BBD688D499D977EB66ED55EF44E133E25
:10192000322E511E700E9FFFBEEFDDDFFCCF1BBFBE
:101930003AAF599F788F8891A981CAB1EBA10CD198
:101940002DC14EF16FE18010A100C230E3200450A0
:10195000254046706760B9839893FBA3DAB33DC313
:101960001CD37FE35EF3B1029012F322D2323542F0
:10197000145277625672EAB5CBA5A89589856EF5A3
:101980004FE52CD50DC5E234C324A0148104667440
:10199000476424540544DBA7FAB79987B8975FE7F3
:1019A0007EF71DC73CD7D326F2369106B016576690
:1019B0007676154634564CD96DC90EF92FE9C8997B
:1019C000E9898AB9ABA94458654806782768C018E0
:1019D000E1088238A3287DCB5CDB3FEB1EFBF98B53
:1019E000D89BBBAB9ABB754A545A376A167AF10A30
:1019F000D01AB32A923A2EFD0FED6CDD4DCDAABD63
:101A00008BADE89DC98D267C076C645C454CA23C7F
:101A1000832CE01CC10C1FEF3EFF5DCF7CDF9BAF32
:101A2000BABFD98FF89F176E367E554E745E932ECF
:101A3000B23ED10EF01E11241FBECFEFD4E0DEBFA8
:101A4000CDBF14BE0FB6F894A89580916000886150
:101A500080936000109260000FBE21E0A0E0B1E032
:101A600001C01D92A13AB207E1F742D278C2C8CEB6
:101A700081E085BF82E085BF089581E085BF15BE06
:101A800008958F929F92AF92BF92CF92DF92EF9282
:101A9000FF920F931F93CF93DF93CDB7DEB7DA9505
:101AA0000FB6F894DEBF0FBECDBF7E0181ECE80E0D
:101AB000F11C8E010F5F1F4FAA24BB24A01AB10A8C
:101AC000D12C470180ECC82EC00ED801FD01EA0DD3
:101AD000FB1DE491ED93CA12F9CFEFE1DE1207C0CE
:101AE0006EEBC801D4D1F40197AF86AF06C060ECAD
:101AF000C801CDD1F70191838083D394F2E0EF0E3A
:101B0000F11C80ECA80EB11CE0E2DE12DECF60E436
:101B1000C401BDD1D3950FB6F894DEBF0FBECDBFC3
:101B2000DF91CF911F910F91FF90EF90DF90CF90B9
:101B3000BF90AF909F908F90089561157105E9F067
:101B4000409105015091060120910301309104015B
:101B500042175307E9F75A9A9C012F5F3F4F309382
:101B6000060120930501680F791F709304016093AB
:101B70000301FC0180818093C60008951F920F929B
:101B80000FB60F9211248F939F93EF93FF93E091E1
:101B90000501F09106018091030190910401E8177D
:101BA000F907B9F4109207015A988091C100806832
:101BB0008093C100809102018823B9F098E088E108
:101BC0000FB6F894A895809360000FBE90936000C4
:101BD000FFCF80818093C60080910501909106011E
:101BE00001969093060180930501FF91EF919F91DB
:101BF0008F910F900FBE0F901F9018951F920F920C
:101C00000FB60F9211248F939F93EF93FF938091C0
:101C100007018D3810F01092070180910701909113
:101C2000C600E82FF0E0E85FFE4F90838F5F80935F
:101C300007011092B1001092B2008AE28093B300C3
:101C400083E08093B10082E08093700010929D0148
:101C5000FF91EF919F918F910F900FBE0F901F906A
:101C600018951F920F920FB60F9211241F932F9366
:101C70003F934F935F936F937F938F939F93AF9314
:101C8000BF93CF93DF93EF93FF9380919D018111D9
:101C90009CC01092B1001092B20092E097BB80916C
:101CA000C1008F778093C1001092B1001092B200F2
:101CB0008AE38093B30083E08093B1009093700037
:101CC00011E010939D01609107016D3008F4A9C0E7
:101CD000862F90E0885F9E4FFC013197C081D0E055
:101CE000DC2FCC2731978081C80FD11D625088E04E
:101CF00091E0CDD08C179D0709F093C0C0910801E9
:101D00008C2F807F803A09F08CC049E050E069E078
:101D100071E080EF90E016D1892B09F082C08C2F02
:101D20008F70863019F4109302014DC0843019F47D
:101D30001093A0015CC0853089F507B600FC54C043
:101D4000809107018E3209F051C020911301203C8F
:101D500008F04CC080E2289F9001112440E050E040
:101D600061E0DA01A85FBE4F1C967C911C97FA01D6
:101D7000E20FF31F1D968C9190E0982F8827870F14
:101D8000911D0C0160935700E89511244E5F5F4F41
:101D90004032510531F785E0F90112C0873031F545
:101DA00007B600FC21C0809107018E30F9F4E09164
:101DB0001301E03CD8F480E2E89FF001112483E0B5
:101DC00080935700E89584E012C08130C1F51092ED
:101DD000B1001092B20082E087BB6091070170E011
:101DE00088E091E0AADE2BC085E001C082E0806D32
:101DF0008093080189E0E0EFF0E0A9E0B1E0019014
:101E00000D928A95E1F7109212016BE088E091E063
:101E10003ED080931301909314018DE080930701CD
:101E20000EC0109207015A988091C100806880937B
:101E3000C1001092B1001092B20082E087BBFF9106
:101E4000EF91DF91CF91BF91AF919F918F917F9152
:101E50006F915F914F913F912F911F910F900FBE06
:101E60000F901F901895529A5A98589AF894109279
:101E7000C5008CE08093C40082E08093C00088EDB0
:101E80008093C10086E08093C20078940895DC01BD
:101E9000762F6A0F8FEF982F40E026E338E150E06D
:101EA0004D914927440F551FF901E40FF51F082EE6
:101EB0008591949190256A1791F70895549A539AB1
:101EC000689A0895CF93DF931F92CDB7DEB78983C9
:101ED000F5DF549A5C9A5398689A898181508230D0
:101EE00010F4709801C0709A0F90DF91CF9108950F
:101EF000BFDDB9DFE3DF82E0E5DFC3DDEEEFF7E171
:101F0000259134912817390721F081E08093A001B1
:101F1000D9DF2FE788E391E0215080409040E1F73E
:101F200000C000008091A0018111FFCFF89480E0F3
:101F3000C9DFA3DDE0910001F0910101099580E086
:101F400090E00895FB01DC0104C08D91019080199F
:101F500021F441505040C8F7881B990B0895F8941C
:021F6000FFCFB1
:0400000300001800E1
:00000001FF
